:040000003EC0F7C047
:10000400FDCFFCCFFBCFFACFBAC1F8CFF7CFF6CFF5
:10001400F5CFF4CFF3CF33C1F1CFF0CFEFCFEECFA5
:10002400EDCFD804F6041405320550056E058C0591
:10003400AA05C805E6050406220640065E067C06F7
:100044009A06B806D606F406120730074E076C0760
:100054006C076C076C076C076C076C076C076C0704
:100064006C07000000001027E80364000A00010088
:1000740000100001100001000000F894EE27ECBB12
:10008400F1E0FBBFEBBFE5BFF8E1F1BDE1BD8DE001
:10009400A2E0BB27ED938A95E9F780E094E0A0E61F
:1000A400ED930197E9F7ECE7F0E0859195910097DE
:1000B40061F0A591B59105901590BF01F0010590EF
:1000C4000D920197E1F7FB01F0CFEFE5EDBFE4E01E
:1000D400EEBFC0E6D1E064C1AF93AFB7AF93BF93B7
:1000E400A8E0B881AA23C9F0AA958894BB1F18F088
:1000F400C09804D0F7CFC09A01D0F4CF000000001C
:100104000000C19A00000000000000000000000090
:10011400C1980000000000000895C098BF91AF91FD
:10012400AFBFAF9121960895249784E0A0E0B0E09A
:10013400E6E6F0E026D28FD1E883E45091D1EA8359
:10014400E881E3508DD1EB83AA81AA3318F0EA81C8
:10015400E75302C0EA81E053EA83AB81AA3318F083
:10016400EB81E75302C0EB81E053EB83EA81EF704C
:10017400EA83FE013396DF01EC91EF70EC93EA81A0
:10018400E295E07FEA83EB81AA81EA2BEA83E0E04F
:10019400E983E881E450A981AE1748F4E98160D18C
:1001A400AA81EA27EA83E981EF5FE983F2CFEA8152
:1001B40024960895C29859D15BD1C29A0000C2987E
:1001C40054D1EBE858D1C29A0000E0E056D108952A
:1001D400000000000000C19A0000000000000000C0
:1001E40000000000C198000000000000089548D1FC
:1001F400BCD100E010E030E0E0E0E093E001C29820
:10020400E0E039D1E0E037D110E0183058F4B39B86
:1002140005C0E02FEE0FE1600E2F01C0000FD8DF04
:100224001F5FF3CFC29A0000043221F0A091DF01D6
:10023400AE3748F0E1E021D1E4E2E0936001E0E090
:10024400E09361010DC0E091DF0128D10083E091CA
:10025400DF01EF5F12D1E091DF0120D1A0E0A083A4
:100264000A3049F4A7DF60DF3E2F303011F4689480
:1002740020F8E0E002D180D1249614D11895EA93B5
:10028400FA93EFB7EA93772051F07A94E42D18D1DA
:10029400E081ECB94394EFE7E41509F44424E991CF
:1002A400EFBFF991E9911895EFE7E715E9F3F894B1
:1002B400772011F45D990BC0E52D02D1A881A083AC
:1002C4005394EFE7E51509F45524739402C0E881CB
:1002D400ECB97894219608952297F6D040D1EF2F67
:1002E400F0E0E983FE013196DF01EC91E06AEC93E2
:1002F400EBD0E491E883C298BBD0ECE6BCD0C29AC0
:100304000000C298E2ECB7D0E0ECB5D0C29A00008D
:10031400C298E981B0D0E881AED0C29A0000C298F8
:10032400E0ECA9D0E0E8A7D0C29A0000C298E0ECC3
:10033400A2D0E1E8A0D0C29A0000C29896D098D08A
:10034400C29A0000C29891D0EBE895D0C29A0000FE
:10035400C298E4EC90D0ECEA8ED0C29A0000C29825
:10036400E8EC89D0E1E987D0C29A0000C298E6ECB3
:1003740082D0EFEB80D0C29A00002296089580D0FC
:10038400E091E001EF5FE093E001A091E001A4308F
:1003940028F0A2DF0FDFE0E0E093E00183D01895BE
:1003A40010E0E0E0E8BBE7E0E7BBEFE3E5BBE0E05B
:1003B400E4BBE2BBE1BBE3BFE2BFEFBDECE0EEBDFB
:1003C400E0E0EDBDECBDE7BDE6BDEAE7EBBDE1E194
:1003D400EABDE0E0E9BDE8BDE2BDE5BDE4BDE3BDE5
:1003E400EBB7E064EBBFE2E0E5BFE0E4EABFE0E1E5
:1003F400E9BFE0E0EBB9E8E4EAB9E6E8E0BDE0E053
:10040400E0BDECE0E9B9E0E8E8B9E0E0E0BFE3B37F
:10041400EF71E093E101C29AE1E0F0E0FA93EA932C
:1004240092D05ADFC7DE789420FE0FC010E013D0BC
:10043400A12FB0E0AE17BF0730F4E12F11D0EA933B
:1004440033DF1F5FF4CFE89420F8EECFFFCF5F9B3C
:10045400FECFECB10895E0E6F1E0FA93EA935EC0D2
:10046400F0E0E05AFE4FE0810895EEECEA9334CEDA
:10047400E9E8EA9331CEEA932FCEE093DF010895C1
:100484000A921A92FA926A937A938A939A93AA9303
:10049400BA93EA93FA93EFB7EA930895F0E0E05A37
:1004A400FE4F0895E991EFBFF991E991B991A991AE
:1004B4009991899179916991F99019900990089588
:1004C400F0E0EE51FE4F0895E091E101A6E2B0E0C4
:1004D400F0E0EE0FFF1FEA0FFB1F0895E1E0F99132
:1004E400F03310F0FA3308F0EE270895E1E0F991C3
:1004F400F03229F0F93010F0FE3008F0EE270895BC
:10050400E1E0F991F05340F0FA3038F0FF75F7501C
:10051400FA3010F0F03108F0EE270895A991B9915E
:10052400EE27FF276D91662311F03196FBCF0895D6
:10053400AA27BB27E991F9910590002011F01196A3
:10054400FBCFFD010895E991F991309639F080EDE2
:1005540097E00197F1F7A8953197C9F708950590A9
:10056400F491E02D08955A934A933A932A931A9357
:100574000A9308955D814C813B812A811981088108
:100584000895AC0FBD1F05900D928A95E1F708956B
:00000001FF
